:020000040000FA
:0400040000EF08F011
:060008000001CED811003A
:10001800D8CF00F0E0CF01F0026E000116D80250F0
:0A00280001C0E0FF00C0D8FF100087
:100040000F017AEC1FF0000102E3D8801200D89073
:100050001200E9CF03F0EACF04F0FACF05F0FBCFAE
:1000600006F082A538D09DA036D09EA034D09E90B8
:10007000CD90F9504544F92603D00CD014D024D0AB
:1000800081A006D0462A090E466425D0452A23D0F1
:10009000466A21D081B01FD0640E446E636B080E97
:1000A000486E452A18D0D89081B0D8804736482E5F
:1000B00012D044C0E9FFEA6A47C0EFFF632B442A2D
:1000C000080E486E452A07D081B002D0450603D0FD
:1000D000456A466A2D8A82A35ED09DA813D09EA849
:1000E00011D09D98A6B905D0A5A903D0A58D2D80C6
:1000F00009D001EE40F09E51E926EFCFADFFA68971
:100100009E2B94079DAA47D09EAA45D0376A096ABC
:10011000ABA203D0AB98AB8832D0ABA409D0AE5021
:10012000010E096EA5AB2BD03B0EAF6EA59B27D061
:10013000AECF07F007BE986B01EE00F09851E926AC
:1001400007C0EFFFA5AB04D03B0EAF6EA59B12D04E
:10015000A6A910D001EE40F09D51E926EFCF08F09E
:100160000750081803E0010E096E04D09D2B9D9BDB
:1001700094679D88096603D02D82982B989BA6A929
:100180000AD0095208E0A6999D98A58D2D80630E8E
:10019000AF6EAD6AA58B05C0FAFF06C0FBFF03C0BA
:1001A000E9FF04C0EAFF120082A509D0F2A807D037
:1001B000F2A205D0F292CF68640ECE6ECD8082A3FB
:1001C00011D0F2A80FD0F2A20DD0F292F298A58928
:1001D000376A2DB007D0A6B905D00D0EA26102D0A6
:0601E000020EA22712002E
:04022E0000EF02F0EB
:0402580000EF02F0C1
:1004000000011EDE03E30D01F4D90001000100EF3D
:1004100008F01200146A1350146009D09E90B10EB7
:10042000CF6ECD809EA0FED7CD90142AF4D71200B7
:10043000898E126A115012600AD0899E0A0E136EBC
:10044000E9DF898E280E136EE5DF122AF3D7C80E76
:10045000136EE0DFEDD70DEE10F000019751E926A5
:10046000EFCF13F00DEE10F0E926EF6A972B400E58
:100470009761976B13500D011200152C02D0176A6B
:10048000000C14C018F0182A1850166201D0186A0F
:100490000D0EEA6E18501324E96EEFCF17F01750C7
:1004A000100A03E0FD0E176EFD0C186A0D0EEA6EC1
:1004B00014501324E96EEF50181A142A14501662BF
:1004C00001D0146A1704196E19521FE0150615BEE3
:1004D00002D0156602D0176A000C0D0EEA6E145099
:1004E0001324E96EEFAE03D0FE0E176EFE0C0D0E58
:1004F000EA6E14501324E96EEF50181A142A14509F
:10050000166201D0146A1906DFD7183C02D01750C2
:1005100012001768FF0C9EAA14D0ABA203D0AB98B0
:10052000AB880FD0ABA402D0AE500BD0899E0DEE9D
:1005300010F09651E926AECFEFFF962B400E966154
:10054000966B9751965D116E11AE02D0400E11263A
:1005500011522BE00DEE10F09751E926E50EEF62F7
:1005600022D0100E136E97C014F011C015F0400E7B
:10057000166E83DF17C091FD0D01915107E0FD0A52
:1005800007E0030A05E0010A06E008D000010DD0EB
:1005900062DF00010AD012680001FF0C898E010E93
:1005A000126E0001010C57DF0001126A000CA6B2A6
:1005B000FED711C0A9FF12C0AAFFA69EA69CA680C6
:1005C000A8501200020E1D6EA69EA69CA68418C0FE
:1005D000A9FF19C0AAFF0DEE00F01BC01CF0EFCF61
:1005E000A8FF550EA76EAA0EA76EA682A6B2FED7CA
:1005F000A680A850EF6209D0020E1D6EEE50A92A07
:10060000A950D8B4AA2A1E8002D01E9002D01C2E57
:10061000E6D71EA002D0D88012001D2EE0D7D890B9
:100620001200899E020E256EA68EA69CA684A68E1A
:1006300020C0F6FF21C0F7FF22C0F8FFA688550EA4
:10064000A76EAA0EA76EA682A6980A000DEE50F01D
:1006500023C024F0EECFF5FF0F00242EFBD7550E5C
:10066000A76EAA0EA76EA682A69420C0F6FF0DEE76
:1006700050F0268023C024F00900F550EE1802E067
:10068000269002D0242EF8D726A004D09281898EFD
:10069000D8801200252ECAD7D8901200A68EA69C0C
:1006A0002250F86E2150F76EC00E2014F66E0DEE3B
:1006B00050F0400E236E0900F5CFEEFF232EFBD73E
:1006C00012003F0E18141F6E500E1F241D6E1D06C3
:1006D0001E6A1F6A1B501F5C1F501B18D8B0800A6F
:1006E00036E61D2A900E1D6219D0500E1D6E93CD58
:1006F00020F094CD21F0226A400E236E92DF0CE3AD
:10070000400E9327000E942393CD20F094CD21F03A
:10071000226AC4DF929102D0D89012000D0EEA6EC8
:100720001EC0E9FFEFCF1CF019501A1003E1030EB1
:10073000186406D00D0EEA6E1DC0E9FF1CC0EFFF65
:100740001E2A182A000E19221A221F2AC3D7D8805F
:1007500012001350176E1250166EC00E1114156E43
:10076000898E175003E1030E166407D0175005E178
:10077000010E155C0A0E16582EE317502CE1F00EF0
:10078000166029D092A10BD015C093FD16C094FD20
:1007900093CD20F094CD21F0226A80DF9291155004
:1007A00093630ED0165094630BD0176609D011C016
:1007B00018F012C019F013C01AF014C01BF081D742
:1007C00093CD20F094CD21F0226A400E236E29DFD4
:1007D000C7E2D8901200F00E136209D011C018F0D1
:1007E00012C019F013C01AF014C01BF0EBD6D88059
:1007F000120092811092899E108000018CDEFF0A07
:100800000D0103E0FE0A07E0C7D010A2C5D0040E18
:10081000116E0EDEC1D0899E1EDE1DDE100AD8A428
:10082000BBD019DE7F0AD8A4B7D015DE7F0AD8A4C2
:10083000B3D011DE7F0AD8A4AFD00DDE0A6E040E4D
:10084000000197250C6E3F0E0C6402D0400E0C5E2A
:100850000DEE10F00C50E926F00EEF140D0108E03B
:10086000100A49E0300A57E0600AD8B486D094D024
:10087000F2DD570A03E0010E116EDADDECDD160A37
:1008800003E0010E116ED4DDE6DD906F909F0AB497
:10089000908F020E000197250C6E3F0E0C6402D063
:1008A000400E0C5E0DEE10F00C50E926EFCF0BF071
:1008B0000D010BA00FD00BB207D09051030A0AE034
:1008C000020E116EB5DD06D0030E906103D0020E4C
:1008D000116EAEDDC0DD906F909F0AB6908F0BA4B5
:1008E00008D0116A126A63DE906103D0030E116EA4
:1008F0009FDD108251D0AFDD0F6E0F9E0AB00F8EBC
:10090000AADD0E6E0E9E0AB20E8EA5DD0D6E0D9E38
:100910000AB40D8E41D01DEE00F00C6A040E0C607E
:1009200009D099DDE76E0A32D8A0E69ED8B0E68EEF
:100930000C2AF4D790DD0B6E0C6A040E0C6009D003
:100940008ADDE76E0B32D8A0E69ED8B0E68E0C2A80
:10095000F4D70DC011F00EC012F00FC013F0080E46
:10096000146EF7DE06E3080E0D26000E0E220F228F
:1009700013D0050E116E5CDD0FD092B10CD093CD6B
:1009800020F094CD21F0226A400E236E4ADE03E26D
:10099000050E116E4DDD109010B02FD7120053BE12
:1009A00009D0D6CF0AF056500A5C575E0AC056F0FE
:1009B000D8A0538E1200D6CF0AF054500A5C555E70
:1009C0000AC054F0D8B012007D0E5526050E0B6EED
:1009D000010E0C6E00EE49F053500C140DE1EF06C1
:1009E000EF3C03D0EE50EF06ED50EF50EE50EF101D
:1009F00002E10C505312ED50020EE926000EEA22DD
:0A0A0000D8900C360B2EE8D7120038
:10100000000103D000EC02F000010D0192A320ECDE
:1010100000F0000121EC20F0A0EC20F048EC21F0E1
:101020005368546A556AC60ED56E2D6A000190EC5D
:1010300021F02D862D88D08EF28EF28C306A316AA6
:10104000326A336A800E436E426E396E3A6E3D6E7E
:101050003E6E3F6E406E416E376E346E356E366E4C
:10106000386E3C6E3B6E356A366A386A3A6A3C6A5C
:101070003B6A0400D19082A505D0346A9E909D8081
:10108000F292F2888CDC97DC30BE02D05CD8306EF5
:1010900031BE02D066D8316E32BE04D002012AD9E8
:1010A000326E000133BE02D085D9336E34BE04D017
:1010B0000101ACD9346E000135BE02D0A4DA356E20
:1010C00036BE02D039DB366E37BE02D060DA376EFC
:1010D00038BE02D0C6DA386E39BE02D08ADB396E2D
:1010E0003ABE02D0A1DB3A6E3BBE03D084EC15F0D1
:1010F0003B6E3CBE03D0DBEC12F03C6E3DBE03D039
:1011000011EC18F03D6E3EBE03D053EC16F03E6E6F
:101110003FBE03D0D9EC16F03F6E40BE03D0A7EC23
:101120001AF0406E41BE03D08DEC1CF0416E42BE01
:1011300003D0A7EC10F0426E43BEA4D70201AFEC7F
:1011400010F0436E9FD7F9503044F92601D004D0F7
:10115000010E496E4A6A539053A0010C6CEC19F0D1
:10116000000CF9503144F92601D004D00A0E4B6E20
:101170004C6A539253A2010C136A020E13603DD0C5
:1011800002EE08F01350E926EFCF10F002EE0AF05D
:10119000E9261050EF14126E02EE10F01350E926FB
:1011A0001050EF140F6E12500F18116E010E0E6ECC
:1011B0000E521BE002EE12F01350E926EF5011140C
:1011C000106E0E5010160EE002EE10F01350E926CD
:1011D0000E50EF1A87B506D002EE18F01350E9262C
:1011E0000E50EF12D8900E36E3D702EE12F01350E5
:1011F000E92611C0EFFF132AC0D73D6A416A3E6A53
:101200003F6A0A6A0B6A2B0EC26EC2B2FED7030E89
:10121000C4140B6EC3CF0AF0120E0A5C010E0B58F9
:1012200003E292EC12F00001130EC26E0C6A0D6A1A
:10123000C2B2FED7030EC4140D6EC3CF0CF0810EE4
:101240000C5C010E0D5814E3800E0C5C020E0D5860
:101250000FE287B318D0070109A303D000018781EB
:1012600002D00001879107010983000187830BD019
:1012700087A309D087A103D00701098302D0070102
:10128000099300018793A5A506D00201022F03D080
:101290000001A595898E0001A5A706D00201052FA2
:1012A00003D00001A597898C000182A322D081B0D0
:1012B00008D0A6A70DD0A02B0A0EA06309D0A69730
:1012C00007D0A06BA6B704D0A16702D0010EA16F12
:1012D000A1530FE0A12B180EA1650BD0A16BF29EBC
:1012E000F292F288AB889E9A9D8A9D98AC8AF28E83
:1012F000A687000C0001F9503244F92601D008D02D
:10130000640E4D6E4E6A5394020153B403D0010C27
:101310000201FBD7000185698669020103530EE0D3
:1013200003070F0E03150AE1033B03070F0E031516
:1013300004E0050E006F426A038B033B045307E091
:10134000042F05D0050E006F426A010E046F0001E4
:1013500082A709D0A5B507D0050E0201006F010EC6
:10136000046F426A0001A5AF21D00B800A6A020E09
:1013700002010A6017D002EE18F00A50E926EF5079
:10138000D8A40B9002EE20F00A50E926EF50D8A422
:101390000B9002EE22F00A50E926EF50D8A40B90F1
:1013A0000A2AE5D70BA002D00001A59F0201000C7C
:1013B0000201800CF9503344F92601D005D0E80E23
:1013C0004F6E030E506E539653A6010CA6A11CD06F
:1013D000A58F02EE08F0A351E926EFCF0AF002EE46
:1013E00018F0E9260A50EF1202EE08F0A351E926A0
:1013F000EF1C0A6E02EE18F0A351E9260A50EF1214
:10140000A32B020EA361A6918795000CF9503444DA
:10141000F92600D02DAA010C20EE63F000EE6FF04B
:101420001F0EDF14866F8629DECFEEFFE806000A66
:10143000FBE12D9A896B010E876F8651876108D079
:10144000EA6A6F0E8725E96EEF50891B872BF5D767
:10145000EA6A6F0E8725E96E8951EF6294D070C0F9
:101460008AF18A4990D0000170AF6BD0050E01015E
:10147000866167D0000171BF2BD03F0E7015040D3F
:10148000F3CF8AF1060E7115D890E83001018A1366
:101490000001711D700BE83A0F0B01018B6F1F0EDD
:1014A00000017215080DF3CF88F1010188518B13EB
:1014B0008A510001856306D001018B5100018663CA
:1014C00001D061D0878B8AC183F08BC184F034D086
:1014D0003F0E7015040DF3CF8AF1070E7115D890E9
:1014E000E83001018A13040E8A5F0001711D700B40
:1014F000E83A0F0B01018B6F010E00017115E83AFC
:10150000F00B0101886F8B138A510001856306D0AF
:1015100001018B510001866301D035D08787829FFE
:101520008AC183F08BC184F0000E9DDA12C00AF0EC
:1015300013C00BF05DEC14F08AC185F08BC186F00E
:10154000406A000170AF1FD0040E010186651BD0F8
:101550003F0E0001701501018B6F71C08AF18A5135
:10156000606303D08B51611906E00F0E8A630BD0C4
:10157000270E8B6308D0EC0E00017215EC0A03E114
:1015800048EC1EF000010101000C0101800CF95033
:101590003744F92602D007D032D0A589D6CF56F0ED
:1015A000960E576E539E53AE010CF292F288A245EE
:1015B0000A6EF9500A44F926960E1DD08E0E1BD0E5
:1015C000860E19D07F0E17D0780E15D0700E13D05E
:1015D000690E11D0610E0FD05A0E0DD0520E0BD0E5
:1015E0004A0E09D0430E07D03C0E05D0340E03D06E
:1015F0002D0E01D0000ED6CF56F0576E539E53AE2F
:10160000020CA599800C0101F9503544F92600D04F
:1016100000012DA2010C436A010100AF1ED054D974
:101620000A6E0A50000119E0FF0A05E10101006B92
:101630000001A69912D011EE00F004EE00F09651D0
:10164000E926E6CFEEFFE950D8B404EE00F00A2E0A
:10165000F8D7E9CF96F0A6992D802D922D8C000118
:10166000000C3850D8A4800C9651971964E004EE11
:1016700000F09751E926EFAE5DD004EE00F0E926C8
:10168000EF50830A0DE0330A0FE0010A22E0030A5B
:101690002FE05F0A3CE0020A46E05B0A49E04AD0DC
:1016A0000701C5EC10F046D04CEC10F00AC083F0F6
:1016B0000BC084F083518415FF0A3CE0000ED3D99F
:1016C00012C00AF013C00BF05DEC14F0829F406A68
:1016D00031D04CEC10F00AC083F00BC084F0835181
:1016E0008415FF0A27E0010EBED9829F406A22D0EE
:1016F0004CEC10F00AC083F00BC084F083518415C9
:10170000FF0A18E0020EAFD9829F406A13D0EDECB9
:101710000FF00AC083F00BC084F083518415FF0AD8
:1017200009E0828F07D00701F7EC1CF0000102D01E
:1017300032EC1FF0972B000C0101F9503644F926CA
:1017400005D004D030D039D040D04ED000012DA4E7
:10175000010C2D94010140390F0B0001A26F0F0EF7
:10176000010140150001946F010E9D6F9E6F82A5CF
:1017700015D09FC098F0586A945158600DD001EE72
:1017800041F05850E926EFCF59F001EE00F0E9267C
:1017900059C0EFFF582AF0D72D8229D0A5B902D021
:1017A000A6B703D0020C0001F9D7D6CF56F095C0EA
:1017B00057F0539E53BE03D0030C0001FBD7436A7E
:1017C0009D882D902DB003D0040C0001FBD7A5AD52
:1017D0000DD0A59DA5B9C3D7D6CF56F095C057F06B
:1017E000539E53BEBCD7050C0001FBD7A26B2D86C0
:1017F000000CF9503944F92600D02DA6010C2D9685
:1018000011EE20F0E6CF0AF021EE40F00AC0DEFF34
:101810000A060B6AE6CFDFFFDE500B1A0A2EFAD754
:101820000B1CDF6E2D84800CF9503A44F92601D050
:1018300006D09B51996303D09C519A1944E02DA680
:10184000010C2D9621EE40F09951E96E050E9A2576
:10185000EA6EEFCF0AF00AC0DEFF992B000E9A2342
:10186000996705D0020E9A6302D0996B9A6B0A06AB
:101870000B6A9951E96E050E9A25EA6EEFCFDFFFEC
:10188000DE500B1A992B000E9A23996705D0020E91
:101890009A6302D0996B9A6B0A2EEBD70B1CDF6E02
:1018A00099519B5D0A6E9A519C590B6E0BAE02D0FA
:1018B000020E0B260BBE05D0D00E0A5C010E0B5893
:1018C000D8A02D882D84000C00AD14D000AB0FD013
:1018D000020E0001986101D0000C01C10BF0030E53
:1018E00001010B6403D0100E0B640BD0FF0C060E2D
:1018F0000B6E07D000AB03D0040E0B6E02D0020EAD
:101900000B6E000198510B6212D00C6A0D6A01EE49
:1019100000F00D50E926EF500C1A0D2A0B500D5C0B
:10192000F6E30C28010102E10B501200FF0C000C41
:10193000176E1438030B186E1B9216BE1B821B9475
:1019400016B81B841BB013D01BA211D017A00FD048
:101950000F0E16141D6E15501C6E1C06000E1D5A1F
:101960001CC015F01DC016F016981BB416881F0E6B
:1019700016161BB019D0185005E0010A06E0030A3C
:101980000AE011D01686169A31D0169A168616A835
:101990002DD016962BD01634163215321698D8B094
:1019A0001688168A23D01200185005E0010A09E0B3
:1019B000030A10E01AD01686100E14BC161A169AD6
:1019C00015D0169A100E14BC161A168616A80ED02C
:1019D00016960CD01634163215321698D8B01688D2
:1019E000168A080E14BC161A01D01200D8901536AB
:1019F0001636D89015329B51E96E050E9C25EA6E7D
:101A0000040EEF6EB7DB9B51E96E050E9C25EA6E66
:101A1000B00E1810EF6EAEDB9B51E96E050E9C25E3
:101A2000EA6E15C0EFFFA6DB9B51E96E050E9C2503
:101A3000EA6E16C0EFFF9EDB99519B5D196E9A51BD
:101A40009C591A6E1AAE02D0020E1A261ABE06D081
:101A5000E10E195C010E1A58D8B02D98050E02013E
:101A6000006F426A12000A6E879D87B7878D0F0E3E
:101A70008415136E8351126E0F6A020E0F60E8D147
:101A80000E68010E106E1052D8B4E0D10E2A02EE8C
:101A900008F00F50E926EF1C1014D8B4D4D10F5021
:101AA000400DF3CFD9FFF4CFDAFF100ED926070E81
:101AB000DA22080E0E02F350D926000EDA220EA00A
:101AC00015D0080ED95E000EDA5ADCCF0BF0DD50CF
:101AD0001C940BBC1C841C960BBE1C861CA602D03E
:101AE0001CA404D0080ED926000EDA22DECF14F092
:101AF000070EDF14156ED9CF1AF0DACF1BF0030EE4
:101B0000D926000EDA22DECF16F0DFCF1DF00F0E41
:101B1000DE14176EDECF18F0DFCF1EF00F0EDE14CE
:101B2000196E1AC0D9FF1BC0DAFFDECF0BF01C9470
:101B30000BBC1C841C960BBE1C86DFCF0CF0DCCFCC
:101B40001FF0DD501F38070B1F6E0B38030B0A62A6
:101B50005ED0125014625BD01350156258D0030E41
:101B60000C1455E01C9284B91C82020EDFBE1C1AB4
:101B70001F50040A03E0060E1F6210D01CB207D0EB
:101B800002EE24F00F50E9261050EF1206D002EEBC
:101B900024F00F50E926101CEF161C82020E0A6278
:101BA0000FD00AC020F0299029921CB229820EC0C1
:101BB00021F00FC022F0105098EC14F0000127D053
:101BC0001CB415D01CA613D00EA011D00AC020F052
:101BD00029901CB4298029821CB229920EC021F0C0
:101BE0000FC022F0105098EC14F0000110D00AC081
:101BF00020F029901CB4298029921CB229820EC0A1
:101C000021F00FC022F0105098EC14F00001030EE8
:101C1000D926000EDA22DFCF0DF0D8900C32D89002
:101C20000C32030E0C14D8B480D01C9284B91C82E0
:101C3000030E0C14010A05E0030A06E0010A06E09F
:101C400074D01CB203D071D01CB26FD00DAE47D08F
:101C5000125016626AD01350176267D0020E0DBC84
:101C60001C1A1F50040A03E0060E1F6210D01CB29B
:101C700007D002EE24F00F50E9261050EF1206D0E4
:101C800002EE24F00F50E926101CEF161C821CB443
:101C900015D01CA613D00EA011D00AC020F0299098
:101CA0001CB4298029821CB229920EC021F00FC0D9
:101CB00022F0105098EC14F0000137D00AC020F048
:101CC00029901CB4298029921CB229820EC021F0CF
:101CD0000FC022F0105098EC14F0000126D01250E2
:101CE000146203D01350151808E0125018621DD06A
:101CF000135019621AD01EAE18D001EE82F00F50A8
:101D0000E926EFCF11F01CA203D01050111202D01F
:101D1000101C111601EE82F00F50E92611C0EFFFE2
:101D200002EE20F0E9261050EF12020ED926000E26
:101D3000DA22DFCF0DF0D8900C32D8900C32030E9F
:101D40000C14D8B480D01C9284B91C82030E0C14DD
:101D5000010A05E0030A06E0010A06E074D01CB29D
:101D600003D071D01CB26FD00DAE47D012501862A4
:101D70006AD01350196267D0020E0DBC1C1A1F5096
:101D8000040A03E0060E1F6210D01CB207D002EE58
:101D900024F00F50E9261050EF1206D002EE24F086
:101DA0000F50E926101CEF161C821CB415D01CA67F
:101DB00013D00EA011D00AC020F029901CB42980A5
:101DC00029821CB229920EC021F00FC022F01050BF
:101DD00098EC14F0000137D00AC020F029901CB410
:101DE000298029921CB229820EC021F00FC022F056
:101DF000105098EC14F0000126D01250146203D059
:101E00001350151808E0125016621DD013501762B7
:101E10001AD01DAE18D001EE84F00F50E926EFCF96
:101E200011F01CA203D01050111202D0101C111678
:101E300001EE84F00F50E92611C0EFFF02EE22F010
:101E4000E9261050EF12D89010361DD60F2A15D65D
:101E5000125012009B51E96E050E9C25EA6E0B0E86
:101E6000EF6E88D99B51E96E050E9C25EA6EED0E4A
:101E7000EF6E80D99B51E96E050E9C25EA6E0B0E24
:101E8000EF6E78D99B51E96E050E9C25EA6E7F0EA8
:101E9000EF6E70D99B51E96E050E9C25EA6E310EEE
:101EA000EF6E68D91438E8441F0B156E143A1442CB
:101EB000F80E1416030E13141412D8901436700E64
:101EC000141A1480149ED8901332D89013329B5158
:101ED000E96E050E9C25EA6E010EEF6E4BD99B5103
:101EE000E96E050E9C25EA6E13C0EFFF43D99B51A6
:101EF000E96E050E9C25EA6E14C0EFFF3BD99B519D
:101F0000E96E050E9C25EA6E15C0EFFF33D99B5193
:101F1000E96E050E9C25EA6EEF6A2CD99B51E96E9D
:101F2000050E9C25EA6EEF6A25D999519B5D156EC9
:101F30009A519C59166E16AE02D0020E162616BE87
:101F400006D0E10E155C010E1658D8B02D98050E7E
:101F50000201006F426A1200136E146882BF04D03F
:101F600087B902D087AB1AD01038E8461F0B1F0B79
:101F7000176E1238E8461F0B1F0B186E070E10164F
:101F800012160F50116227D01050126224D0146A1A
:101F90001750186220D0010E146E1DD01038030B9C
:101FA000176E1238E840E8423F0B030B186E1750CB
:101FB000186211D0070E10161214166E1150156EFD
:101FC0000F50156208D01050166205D0146A12B86E
:101FD000142A1350141A14501200972B04EE00F018
:101FE0009751E926EF500B0A03E00A680B68FF0CD3
:101FF000972B04EE00F09751E926EF507F0A03E09B
:102000000A680B68FF0C972B04EE00F09751E92645
:10201000EF38070B030A03E00A680B68FF0C972BE5
:1020200004EE00F09751E926070EEF14010A03E0D1
:102030000A680B68FF0C972B04EE00F09751E92615
:10204000EFCF0AF00AAC03D00A680B68FF0CD890F7
:102050000A36D8900A36972B04EE00F09751E926FD
:10206000EFCF0BF0700E0B1AD8900B32030E0B143F
:102070000A120B3A0B461F0E0B16972B04EE00F0BC
:102080009751E926EFCF0CF00C3A0C42F80E0C16E3
:102090000C500B120A50120004EE00F09751E92682
:1020A000EFCF0CF0972B04EE00F09751E926D89073
:1020B000EF340A6E972B04EE00F09751E926EFCF2C
:1020C0000DF004EE00F0E9263F0EEF140B6E0E90BB
:1020D0000DBC0E80030E0C14020A05E0030A0DE08D
:1020E000010A1EE032D00EB003D00A680B68FF0C64
:1020F0000A900DBA0A800B8E28D00EB00BD00DBA04
:1021000002D00DA804D00DAA05D00DA803D00A68EE
:102110000B68FF0CD8900B320A320B960B8C15D043
:102120000EA003D00A680B68FF0CD8900B320A325D
:102130000BB60AD00AC00FF00BC010F007012CD864
:102140000A680B680001FF0C0B960A5012004250FF
:10215000D8A4800C00C202F2A585899E800C435051
:102160000001D8A4800C020E0201056F0001A587B2
:10217000899C800C9B2B000E9C239B6705D0020E34
:102180009C6302D09B6B9C6B120009A503D00001DD
:10219000A36BA68100011200070E1014166E0F50DB
:1021A000156EF80E155C030E1658D8A0D2D0FC0E92
:1021B000155C030E1658D8B0CCD0030E0F14146E55
:1021C00010B81484116A020E1160BED01268010E9C
:1021D000136E1352D8B4B6D0122A1150400DF3CF5B
:1021E000D9FFF4CFDAFF100ED926070EDA22080E37
:1021F0001202F350D926000EDA22DECF17F0DF38B4
:10220000030B196E0F0EDE14186E18BC98D0030E57
:102210001C6ED890183217321C2EFBD7186A070E86
:102220001716DECF1AF01B901ABC1B80030E1A146F
:102230001BE01750146218D009A70AD01BA008D0C1
:10224000195206E002EE18F01150E9261350EF1271
:1022500009A90AD01BB008D0196606D002EE18F002
:102260001150E9261350EF12DE50DECF17F0DF38A1
:102270000F0B196E1B9019B61B80030E19160F0E4B
:10228000DE14186E030E1C6ED890183217321C2EF6
:10229000FBD7186A070E17160C0E1A141BE01750FE
:1022A000146218D009A70AD01BB008D0195206E052
:1022B00002EE20F01150E9261350EF1209A90AD0BE
:1022C0001BA008D0196606D002EE20F01150E926B6
:1022D0001350EF12DECF17F0DF380F0B196E1B9083
:1022E00019B61B80030E19160F0EDF14186E030E9D
:1022F0001C6ED890183217321C2EFBD7186A070EA6
:102300001716300E1A141BE01750146218D009A7C4
:102310000AD01BB008D0195206E002EE22F011508C
:10232000E9261350EF1209A90AD01BA008D019669C
:1023300006D002EE22F01150E9261350EF12D89089
:10234000133647D7112A3FD7180E091502E00001AE
:10235000A58F070112001B6E020EEA6E1AC0E9FF7C
:102360001B461B46F9501B44F926EF6A000E00007D
:102370003BD00A0EEF6E000E37D0140EEF6E000E3B
:1023800033D0230EEF6E000E2FD0320EEF6E000E04
:102390002BD0410EEF6E000E27D0500EEF6E000EC8
:1023A00023D0640EEF6E000E1FD07D0EEF6E000E78
:1023B0001BD0960EEF6E000E17D0C80EEF6E000EFB
:1023C00013D02C0EEF6E010E0FD0900EEF6E010E9B
:1023D0000BD0F40EEF6E010E07D0580EEF6E020E0A
:1023E00003D0200EEF6E030EEC6E12001B6E020E79
:1023F000EA6E1AC0E9FF1B461B461B44060FF92470
:10240000D8B0FA2AF96EE80EEF6E030E3BD0DC0E60
:10241000EF6E050E37D0D00EEF6E070E33D0B80E2C
:10242000EF6E0B0E2FD0A00EEF6E0F0E2BD0880E7E
:10243000EF6E130E27D0700EEF6E170E23D0280EFE
:10244000EF6E230E1FD0E00EEF6E2E0E1BD0500E3F
:10245000EF6E460E17D0C00EEF6E5D0E13D0300E2D
:10246000EF6E750E0FD0A00EEF6E8C0E0BD0100E0F
:10247000EF6EA40E07D0800EEF6EBB0E03D0600E81
:10248000EF6EEA0EEC6E12001B6E020EEA6E1AC0C0
:10249000E9FF1B461B461B44060FF924D8B0FA2A55
:1024A000F96E050EEF6E000E3BD00A0EEF6E000EB9
:1024B00037D0140EEF6E000E33D0230EEF6E000EE9
:1024C0002FD0320EEF6E000E2BD0410EEF6E000EAD
:1024D00027D0500EEF6E000E23D0640EEF6E000E6C
:1024E0001FD07D0EEF6E000E1BD0960EEF6E000E0D
:1024F00017D0C80EEF6E000E13D02C0EEF6E010E2B
:102500000FD0900EEF6E010E0BD0F40EEF6E010E99
:1025100007D0580EEF6E020E03D0200EEF6E030EA2
:10252000EC6E120082B91CD0070109A119D0F29EED
:10253000900E0E6E010E0F6E0EC014F00FC015F04F
:10254000020110514AEC1FF00E2A000E0F220EC09D
:1025500014F00FC015F011514AEC1FF000018289F0
:10256000116A126A2B0EC26E0001C2B2FED7030EB0
:10257000C414126EC3CF11F01D0E115C010E12585F
:1025800009E2899E640E146E08D8898E640E146E5A
:1025900004D8E6D7D190FF001200156A14501560D8
:1025A00009D0A192B10EB36EB180A1A2FED7B190B5
:1025B000152AF4D71200F9503C44F92602D006D06F
:1025C0002FD05C6A020E5C6041D1010C02EE18F063
:1025D0005C50E926EF50D8B437D102EE08F05C50D9
:1025E000E926EF50D8B430D15A68010E5B6E5B52C9
:1025F000D8B42AD15A2A02EE18F05C50E926EFCF5F
:102600005DF002EE08F0E926EF505D165B505D14B8
:10261000D8B417D102EE18F05C50E9265B1CEF1617
:102620002DA8020C5C50400DF3CFD9FFF4CFDAFF98
:10263000100ED926070EDA22080E5A02F350D926B8
:10264000000EDA22DECFA7F0A86BDFCFA8F0DECF36
:102650000AF0DFCF0BF0DECF0CF0DECF0DF002EE94
:1026600010F05C50E9265B50EF14A889D8B4A89903
:10267000A7C05EF0A8C05FF00A38030B03E1A5AF66
:1026800064D0DFD00D38070B60E1A5BF5ED002EE4D
:102690000CF05C50E9265B50EF1416E002EE0CF0F3
:1026A0005C50E9265B1CEF1602EE1AF05C50E9263E
:1026B0005B50EF14D880D8B4D89003E2A8B9C1D049
:1026C00044D0A8B942D0BDD002EE1EF05C50E9263D
:1026D0005B50EF1424E102EE1AF05C50E9265B1C1B
:1026E000EF16A8A913D002EE1AF05C50E9265B5051
:1026F000EF12030E0C14030A28E00DC00FF05AC0AD
:1027000010F05CC011F05B50A2D89BD00DC00FF050
:102710005AC010F05CC011F05B5099D892D002EE14
:102720001AF05C50E9265B50EF14D880D8B4D890EA
:1027300003E2A8B903D009D0A8B907D002EE1EF071
:102740005C50E9265B1CEF167CD0030E0C14010ACA
:1027500007E0030A08E0010A08E0030A38E005D0B0
:10276000A8B903D034D0A8B932D002EE16F05C502C
:10277000E926EFCF0EF0A8AD03D05B500E1A08D0BB
:10278000A8B902D05B1C0E16A8A902D05B500E128D
:102790005B500E14A889D8B4A89902EE16F05C50CC
:1027A000E9260EC0EFFF000EA8B9010E0BAE04D053
:1027B000000AA899D8B4A8890AC014F01B90A7C031
:1027C00015F0A8C016F05A5098EC0CF000015EC04D
:1027D000A7F05FC0A8F0A5BF34D0D8900C32D89035
:1027E0000C32030E0C14010A07E0030A08E0010A88
:1027F00008E0030A0CE005D0A8B903D008D0A8B9B6
:1028000006D002EE20F05C50E9265B50EF12D89023
:102810000C32D8900C32030E0C14010A07E0030AA4
:1028200008E0010A08E0030A0CE005D0A8B903D0CB
:1028300008D0A8B906D002EE22F05C50E9265B5021
:10284000EF12D8905B36D3D65C2ABCD6000C126E41
:102850000F0E0F14136E0F38070B146E020A02E0EE
:1028600014662AD0080E1102F3501024156E13526C
:1028700007E0D8901534260F1A6E13506CDD16D071
:10288000020E146209D002EE26F0D8901534E92623
:102890000A0EEE6EEF6A0AD0146608D002EE26F039
:1028A000D8901534E926010EEE6EEF6A02EE1EF0A6
:1028B0001150E9261250EF1212000A500B14FF0AB1
:1028C0000001D8B4120027EE10F0116A020E116058
:1028D0002ED00F6A010E106E105227E0DECF0CF0E2
:1028E000DFCF0DF00DBE19D0070E0D16DECF0EF0A6
:1028F000129084B912800E38030B0FE10A500C625B
:102900000CD00B500D6209D02C9012B02C80140EFC
:1029100011242A6E10505AEC19F0060ED926000E1A
:10292000DA220F2AD8901036D7D7112ACFD7120023
:10293000236E020129B013D02C9029B22C80100EE6
:1029400022242A6E23505AEC19F002EE18F022507D
:10295000E9262350EF12050E006F426AD4D020669C
:10296000D2D021B007D002EE1EF02250E926231C5F
:10297000EF1608D002EE1EF02250E926D890233040
:10298000FF0AEF1621B027D02C8029B22C90100E10
:1029900022242A6E23505AEC19F02C8029B22C9054
:1029A0000E0E22242A6E23505AEC19F02C9029B2D4
:1029B0002C80100E22242A6ED89023345AEC19F061
:1029C0002C9029B22C800E0E22242A6ED89023340B
:1029D0005AEC19F098D029B21FD02C90100E222456
:1029E0002A6E23505AEC19F02C900E0E22242A6ED7
:1029F00023505AEC19F02C90100E22242A6ED890F5
:102A000023305AEC19F02C900E0E22242A6ED89006
:102A100023305AEC19F077D0D9CF27F0DACF28F04D
:102A20002250400DF3CFD9FFF4CFDAFF130ED92691
:102A3000070EDA22080E2102F350D926000EDA2200
:102A40000F0EDF14256E255006E0050A04E00F0A7C
:102A500002E0050A27E12C9025B22C80100E2224DA
:102A60002A6E23505AEC19F02C9025B22C800E0EB1
:102A700022242A6E23505AEC19F02C9025B02C8079
:102A8000100E22242A6ED89023305AEC19F02C9084
:102A900025B02C800E0E22242A6ED89023305AECBA
:102AA00019F02DD02C80100E22242A6E23505AECBF
:102AB00019F02C80100E22242A6ED89023305AEC64
:102AC00019F0080ED95E000EDA5A5F0EDF1417E017
:102AD000060E2114266E080E2202F3502624246EC0
:102AE00002EE26F0D8902434E926010EEE6EEF6A4D
:102AF00002EE1EF02250E926D8902330EF1227C0B4
:102B0000D9FF28C0DAFF1200F9503B44F92602D061
:102B10001AD030D0AA6B020EAA61C4D002EE18F00F
:102B2000AA51E926EFCFACF002EE08F0E926EF1C3F
:102B3000AC15D8B4B5D0A969010EAB6FAB53D8B4FE
:102B4000AFD0A92B010C02EE18F0AA51E926EFCF65
:102B5000ACF002EE08F0E926EF1CAC17AB51AC1557
:102B6000D8B49BD002EE18F0AA51E926AB1DEF169F
:102B7000A5AF39D02DA8020CAA51400DF3CFD9FF33
:102B8000F4CFDAFF110ED926070EDA22080EA903B8
:102B9000F350D926000EDA22DDCF0BF00BBC7DD02E
:102BA0000B38030B7AE1DECF0CF00D6ADECF0DF0AF
:102BB00002EE10F0AA51E926AB51EF140D88D8B4FB
:102BC0000D98DFAE04D0000A0D98D8B40D88100E11
:102BD000146E1B900CC015F00DC016F0A95198ECA6
:102BE0000CF000015AD0AA51400DF3CFD9FFF4CF19
:102BF000DAFF110ED926070EDA22080EA903F350C8
:102C0000D926000EDA22DECFADF0DECFAEF0DECF79
:102C1000AFF00F0EAF15B06FAF39070BAF6F030EEC
:102C2000AE150CE0AFC010F0B0C011F0ADC012F0A6
:102C3000A9C013F0AAC014F0AB5141D9DCCF0AF0FF
:102C4000D890AE33D890AE33030EAE150EE00AAE78
:102C50000CD0AFC010F0B0C011F0ADC012F0A9C0E0
:102C600013F0AAC014F0AB512AD9DE50DCCF0AF021
:102C7000D890AE33D890AE33030EAE150EE00AAE48
:102C80000CD0AFC010F0B0C011F0ADC012F0A9C0B0
:102C900013F0AAC014F0AB5112D9D890AB374ED76D
:102CA000AA2B39D7000CF9503E44F92602D012D095
:102CB0001FD0B36B020EB3617BD002EE20F0B35194
:102CC000E926EF5073E0B169010EB26FB2536EE0C6
:102CD000B12B010C02EE18F0B351E926B251EF14FA
:102CE00062E102EE20F0B351E926B251EF145BE04D
:102CF0002DA8020C02EE20F0B351E926B21DEF160A
:102D0000B351400DF3CFD9FFF4CFDAFF100ED9261F
:102D1000070EDA22080EB103F350D926000EDA228C
:102D2000DCCF0AF0030ED926000EDA22DECF0BF03C
:102D30000C6A3F0EDF140C6EDFCF0DF001EE82F057
:102D4000B351E926B251EF140C88D8B40C980E9008
:102D50000ABE0E8002EE08F0B351E926B251EF141C
:102D60000EE00EB00CD00A38030B09E102EE14F0AD
:102D7000B351E926B251EF140C88D8B40C98A5AF22
:102D800007D00D38030B0F6E0F6602D0100E0D6EBC
:102D90000DC014F01B800BC015F00CC016F0B15123
:102DA00098EC0CF00001D890B23790D7B32B82D7B3
:102DB000800CF9503F44F92602D012D01FD0B56BD9
:102DC000020EB5617BD002EE22F0B551E926EF503C
:102DD00073E0B669010EB46FB4536EE0B62B010C0C
:102DE00002EE18F0B551E926B451EF1462E102EE9B
:102DF00022F0B551E926B451EF145BE02DA8020C86
:102E000002EE22F0B551E926B41DEF16B551400D82
:102E1000F3CFD9FFF4CFDAFF100ED926070EDA224E
:102E2000080EB603F350D926000EDA22DCCF0AF0E2
:102E3000050ED926000EDA22DECF0BF00C6A3F0E0B
:102E4000DF140C6EDFCF0DF001EE84F0B551E926F2
:102E5000B451EF140C88D8B40C980E900ABE0E80B2
:102E600002EE08F0B551E926B451EF140EE00EB0B1
:102E70000CD00A38030B09E102EE14F0B551E92633
:102E8000B451EF140C88D8B40C98A5AF07D00D3806
:102E9000030B0F6E0F6602D0100E0D6E0DC014F0F6
:102EA0001B800BC015F00CC016F0B65198EC0CF05E
:102EB0000001D890B43790D7B52B82D7800C156E0F
:102EC00002EE10F01450E9261550EF14D8B48DD04E
:102ED000080E1402F3501324166E105203E0020E73
:102EE000106208D0D8901634260F1A6E1150ABEC31
:102EF00011F01AD0104C03D0030E106208D0D890F5
:102F00001634260F1A6E1150F6EC11F00DD0105039
:102F1000040A03E0060E106207D0D8901634260F7C
:102F20001A6E115044EC12F002EE26F0D8901634CE
:102F3000E926EECF18F0EECF19F01050020A0BE0A0
:102F4000010A14E0050A12E0060A2DE0010A36E043
:102F5000050A34E048D01850191008E102EE0EF0CE
:102F60001450E9261550EF12D890120002EE1EF010
:102F70001450E9261550EF1436E102EE0EF014500D
:102F8000E9261550EF1A02EE26F0D8901634E926FD
:102F900018C0EEFF19C0EEFF02EE1EF01450E92635
:102FA0001550EF1220D01850191008E102EE0EF063
:102FB0001450E9261550EF12D890120002EE0EF0D0
:102FC0001450E9261550EF1202EE26F0D890163470
:102FD000E92618C0EEFF19C0EEFF02EE1EF01450F5
:102FE000E9261550EF12D88012001050020A0BE0AB
:102FF000010A09E0050A07E0060A0BE0010A09E0F8
:10300000050A07E00CD002EE1EF01450E926151C4C
:10301000EF1602EE0EF01450E926151CEF16D890AC
:103020001200F9503D44F92601D005D0B76B020ECD
:10303000B761B4D0010C02EE1EF0B751E926EF5093
:10304000D8B4AAD00B68010E0A6E0A52D8B4A4D024
:103050000B2A02EE1EF0B751E9260A50EF14D8B43D
:1030600098D0B751400DF3CFD9FFF4CFDAFF100E4F
:10307000D926070EDA22080E0B02F350D926000ECD
:10308000DA22DCCF0CF0DCCF0EF0DCCF0DF00D3807
:10309000070B0F6E02EE26F0080EB703F3500B2459
:1030A000D890E834E926EE06000EEF5A02EE26F03C
:1030B000080EB703F3500B24D890E834E926EE50FD
:1030C000EF1067E102EE08F0B751E926EF1C0A1491
:1030D0004EE00CAC19D0080ED926000EDA220D38BD
:1030E000F00B0D6E0F0EDF140D26080ED95E000ECC
:1030F000DA5A0FC010F00DC011F00BC012F0B7C0BB
:1031000013F00A504CD845D00F50020A06E00F5079
:10311000030A03E0060E0F6213D002EE1EF0B75151
:10312000E9260A1CEF160FC010F00F0E0D14116ED9
:10313000126A0BC013F0B7C014F00A50C0DE14D0EE
:103140000F5205E00F4C03D0040E0F620DD002EEBB
:103150001EF0B751E9260A1CEF1602EE0EF0B75129
:10316000E9260A1CEF1615D0A5AF13D012D002EE37
:103170001EF0B751E9260A1CEF1602EE0CF0B7510B
:10318000E9260A50EF1202EE18F0B751E9260A506C
:10319000EF12D8900A3659D7B72B49D7800C146E46
:1031A00002EE0EF01350E926196AEFCF18F0125014
:1031B00005E01A6ED89018321A2EFCD7196A030E41
:1031C00018161114186212D02C9011B42C800E0E07
:1031D00013242A6E14506ED82C9011B62C800E0E2B
:1031E00013242A6ED890143465D811D02C9011B0C5
:1031F0002C800E0E13242A6E14505CD82C9011B221
:103200002C800E0E13242A6ED890143453D8113803
:103210000F0B116E080E1302F3501224156E02EEFE
:103220001EF01350E926141CEF161050020A05E098
:10323000010A1DE0050A1BE033D0D8901534260F93
:103240001A6E1150ABEC11F002EE26F0D890153446
:10325000E926EECF16F0EECF17F01650171020E04B
:1032600002EE1EF01350E9261450EF1219D0D89038
:103270001534260F1A6E1150F6EC11F002EE26F0FE
:10328000D8901534E926EECF16F0EECF17F0165091
:10329000171006E002EE1EF01350E9261450EF124C
:1032A00002EE26F0D8901534E92616C0EEFF17C0BE
:1032B000EEFF12002B6E020EEA6E2AC0E9FFD890D4
:1032C0002B50EF14D8A4D8802CA003D02B50EF1291
:1032D00002D02B1CEF1612000A6A020E0A6036D1C9
:1032E00002EE0EF00A50E926EFCF0BF002EE08F0E6
:1032F000E926EF1C0B1602EE1CF00A50E926EF50EF
:103300000B1A0A6691D002EE08F00A50E926EFB0D7
:1033100005D00BA08A960BB08A8607D002EE0AF081
:103320000A50E926EF9081B6EF8002EE08F00A50CD
:10333000E926EFB205D00BA289960BB2898607D099
:1033400002EE0AF00A50E926EF9280B6EF8202EE12
:1033500008F00A50E926EFB405D00BA48A940BB408
:103360008A8407D002EE0AF00A50E926EF9481B46D
:10337000EF8402EE08F00A50E926EFB605D00BA65E
:1033800089940BB6898407D002EE0AF00A50E92628
:10339000EF9680B4EF8602EE08F00A50E926EFB807
:1033A00005D00BA88B920BB88B8207D002EE0AF0E7
:1033B0000A50E926EF9882B2EF8802EE08F00A5030
:1033C000E926EFBA05D00BAA89920BBA898207D0F9
:1033D00002EE0AF00A50E926EF9A80B2EF8A02EE76
:1033E00008F00A50E926EFBC05D00BAC8B900BBC63
:1033F0008B8007D002EE0AF00A50E926EF9C82B0DB
:10340000EF8C02EE08F00A50E926EFBE05D00BAEB5
:1034100089900BBE898098D002EE0AF00A50E92606
:10342000EF9E80B0EF8E90D002EE08F00A50E926B1
:10343000EFB005D00BA08B9A0BB08B8A07D002EEB1
:103440000AF00A50E926EF9082BAEF8002EE08F007
:103450000A50E926EFB205D00BA28A9E0BB28A8EE3
:1034600007D002EE0AF00A50E926EF9281BEEF8201
:1034700002EE08F00A50E926EFB405D00BA48B98B1
:103480000BB48B8807D002EE0AF00A50E926EF94BD
:1034900082B8EF8402EE08F00A50E926EFB605D0B4
:1034A0000BA68A9C0BB68A8C07D002EE0AF00A5053
:1034B000E926EF9681BCEF8602EE08F00A50E92675
:1034C000EFB805D00BA88B960BB88B8607D002EE11
:1034D0000AF00A50E926EF9882B6EF8802EE08F06B
:1034E0000A50E926EFBA05D00BAA8A9A0BBA8A8A43
:1034F00007D002EE0AF00A50E926EF9A81BAEF8A65
:1035000002EE08F00A50E926EFBC05D00BAC8B9414
:103510000BBC8B8407D002EE0AF00A50E926EF9C20
:1035200082B4EF8C02EE08F00A50E926EFBE05D017
:103530000BAE8A980BBE8A8807D002EE0AF00A50BA
:10354000E926EF9E81B8EF8E0A2AC7D61200F950FD
:103550004044F92602D0E3D055D1800E386E2C9825
:10356000B86B200EB86150D1080EB803F350900F1D
:10357000B96F070EBA6BBA23B9C0D9FFBAC0DAFF68
:10358000DFAE40D1040ED924E16E000EDA20E26EE7
:103590002C96E6CF0BF0E7CF0CF00D6AE7BC0D2AB6
:1035A0000E90E7B80E80DFB802D0E7AE3DD0DFA8BE
:1035B00004D082BF08D087BB06D0DFB83AD082AF34
:1035C00002D087AD36D00C980BC00FF00CC010F0B5
:1035D00083C011F084C012F00D50ACEC0FF014C099
:1035E0000AF00ABE26D001EE62F0B851E926EF9C3F
:1035F0000AB00CD001EE62F0E926EF9A0AB0EF8A29
:1036000001EE62F0E926EF900AB0EF8001EE62F081
:10361000B851E926EF900AB0EF800EA00AD001EE73
:1036200062F0E926EF8C05D001EE62F0B851E92690
:10363000EF80060ED924E16E000EDA20E26EE6CFAE
:103640000BF0E7CF0CF00D6AE7BC0D2A0E90E7B83F
:103650000E80DFB602D0E7AE34D0DFA604D082BF42
:1036600008D087BB06D0DFB631D082AF02D087AD9D
:103670002DD00C980BC00FF00CC010F083C011F0CF
:1036800084C012F00D50ACEC0FF014C00AF00ABE6A
:103690001DD001EE62F0B851E926EFA004D001EE92
:1036A00062F0E926EF8A01EE62F0B851E926EF9266
:1036B0000AB0EF820EA00AD001EE62F0E926EF8C8C
:1036C00005D001EE62F0B851E926EF820E92DFBC20
:1036D0000E822CB806D0B8519BD82C96D8B02C8628
:1036E00009D001EE62F0B851E926EF9801EE62F0E0
:1036F000E926EF9601EE62F0B851E926EFB62C8884
:103700000EB22C982CA67DD0D9CFE1FFDACFE2FF04
:10371000E4BE05D001EE62F0E926EFB872D02DA824
:10372000010CB9C0D9FFBAC0DAFFD9CFE1FFDACFB7
:10373000E2FF070EE4140FE0010A11E0030A13E0B0
:10374000010A15E0070A17E0010A19E0030A1CE064
:10375000010A1FE022D0010E0A6E0B6A1ED0050E70
:103760000A6E0B6A1AD00A0E0A6E0B6A16D0320E57
:103770000A6E0B6A12D0640E0A6E0B6A0ED0F40E3B
:103780000A6E010E0B6E09D0E80E0A6E030E0B6E68
:1037900004D0880E0A6E130E0B6EE738E8461F0B36
:1037A0000F0B0C6E0A500C02F3CF0DF0F4CF0EF09D
:1037B0000F6A0B500C02F3500E26F4500F220CAE81
:1037C00004D00A500E5E0B500F5A0BAE02D00C50B4
:1037D0000F5E0D500E100F1012E003EE00F0030EFE
:1037E000B803F350E9260DC0EEFF0EC0EEFF0FC088
:1037F000EEFF01EE62F0B851E926EF8802D0B85131
:10380000BDD8020CB82BADD6879B879D386A800C3B
:103810000F6E1190080E0F02F350900FE16E070E1D
:10382000E26AE22201EE62F00F50E926D890E7301A
:1038300006E3EFB002D0EFA206D0118004D0EFA0D3
:1038400002D0EFB21180D890E730030B106E105009
:1038500007E0010A1DE0030A33E0010A41E05BD002
:1038600011A013D0EFBC07D011B003D0EFB403D038
:1038700007D0EFB405D0EF86EF84EF9CD88012001C
:10388000EFB649D0EF86D8801200EF96EF9443D080
:1038900011B013D0EFBC07D011B003D0EFB403D0F8
:1038A00007D0EFB405D0EF86EF94EF9CD8801200DC
:1038B000EFB631D0EF86D8801200EF96EF842BD090
:1038C000EFBC07D011B003D0EFB403D024D0EFB4D5
:1038D00022D011A0EF9411B0EF84EF9CD880120099
:1038E00011A017D0EFBA02D0D8901200EFBC07D0C9
:1038F00011B003D0EFB403D007D0EFB405D0EF86FA
:10390000EF84EF9CD8801200EFB605D0EF86D88008
:103910001200EF96EF94D8901200F9504144F92626
:1039200002D006D024D0BB6B200EBB6126D0010C88
:1039300001EE62F0BB51E926EFA81DD003EE00F0C6
:10394000030EBB03F350E926EE06000EEE5AEF5AC3
:1039500003EE00F0030EBB03F350E926EE50EE1029
:10396000EF1009E101EE62F0BB51E926EF982DA8B6
:10397000020CBB5103D8BB2BD7D7800C106E080E9E
:103980001002F350900FE16E070EE26AE222E7AAFE
:1039900013D0020EE126000EE222E6CF11F0126AE9
:1039A000E7CF12F00B0E9F6F11C013F012C014F08E
:1039B0002AEC0FF000011AD0020EE126000EE222DE
:1039C000E6CF11F0126A0F0EE714126E1288E7CFDD
:1039D00013F0040E9F6F13C014F01B8011C015F07C
:1039E00012C016F0000E98EC0CF00001120009A3B2
:1039F00012000001972B972B04EE00F09751E92657
:103A00007C0EEF625CD0972B04EE00F09751E92614
:103A1000EFCF0CF0972B972B04EE00F09751E9268F
:103A2000EFCF0BF0972B04EE00F09751E926D890DA
:103A3000EF340A6E0B340B320A320A500101606314
:103A400004D00B50616301D00BD0000187A307D0D5
:103A50000F0E0A6204D0270E0B6201D001D01200B3
:103A60000001972B972BFC0E0C14200A0BE0080A80
:103A700009E0040A11E04C0A19E0080A17E00C0AF0
:103A80001AE01DD00CC00DF00AC00EF00BC00FF0F4
:103A900017D8010EAFD913D00CC00DF00AC00EF02C
:103AA0000BC00FF00DD8010EA5D909D0F1D8400EEA
:103AB0000001A0D904D0ECD8400E00019BD912001F
:103AC00011EE20F00E0EE66EE70EE66E0E0EE66EBE
:103AD0007C0EE66E0DC0E6FFE66AD8900E360F3615
:103AE000D8900E320FC0E6FF0EC0E6FFE66A166AF7
:103AF00004EE00F09751E926EFCF14F014C013F054
:103B000013380F0B136E972B04EE00F09751E92634
:103B1000EFCF15F015C012F0129E14B0128E179050
:103B2000125013100AE1040E126E136AE96E070EAA
:103B30001324EA6EEFCF16F01780135003E1050E41
:103B4000126412D0135010E1090E12600DD0060E4F
:103B5000125E000E135A1250E96E070E1324EA6E1D
:103B6000EFCF16F017807FD0100E126202D01352E2
:103B700005E0110E12620FD013660DD00C0E125E0E
:103B8000000E135A1250E96E070E1324EA6EEFCF9F
:103B900016F0178068D01B0E126202D0135205E097
:103BA0001C0E12620FD013660DD0150E125E000EA1
:103BB000135A1250E96E070E1324EA6EEFCF16F077
:103BC000178051D06F0E126214D0136612D0660E99
:103BD000125E000E135A1250E96E070E1324EA6E9D
:103BE000EFCF16F087A303D0169287B11682178005
:103BF0003AD0135003E16F0E126412D0135010E14B
:103C0000730E12600DD0660E125E000E135A125023
:103C1000E96E070E1324EA6EEFCF16F0178023D05B
:103C2000135002E112AE10D013660ED0800E125E59
:103C3000000E135A100E1224E96E070E1320EA6EBE
:103C4000EFCF16F017800FD013520DE0020E136065
:103C50000AD01306900E1224E96E070E1320EA6EA6
:103C6000EFCF16F01780149216BE148214C0E6FF30
:103C700015C0E6FF7F0E1614E66EE66AE66A17A028
:103C800005D0050E0201006F426A0001A68B1200EA
:103C9000119082A50CD00C0E72150C0AD8A412003B
:103CA000030E7215106E73C00FF074C00DF082A376
:103CB0001DD004EE00F09751E926EFCF10F0972BBE
:103CC00004EE00F09751E926EFCF0FF00F9E10B0F1
:103CD0000F8E972B04EE00F09751E926EFCF0DF0F1
:103CE0000D9E10B20D8E10380F0B106E10502FE17C
:103CF000200E0F602CD0100E0F6202D0105205E083
:103D0000110E0F620ED010660CD00C0E0F5E000E5E
:103D1000105A0F50E96E070E1024EA6E0DC0EFFF27
:103D200058D01B0E0F6202D0105205E01C0E0F621D
:103D300050D010664ED0150E0F5E000E105A0F5068
:103D4000E96E070E1024EA6E0DC0EFFF42D06F0E31
:103D50000F6213D0106611D0660E0F5E000E105A5F
:103D60000F50E96E070E1024EA6E800E0D10EF6EF4
:103D700087910DB2878111802CD0105002E10FAED7
:103D800014D0106612D0800E0F5E000E105A100E66
:103D90000F24E96E070E1020EA6E0DC0EFFF100E23
:103DA0000F26000E1022118014D0105211E0020EC6
:103DB00010600ED01006900E0F24E96E070E102032
:103DC000EA6E0DC0EFFF900E0F26000E102201D0FC
:103DD00012000FC014F010C015F00D505BD811A0E8
:103DE00004D0AED955DA00019BDA050E0201006F4E
:103DF000426A12000D6E9B51E96E050E9C25EA6E1B
:103E0000040EEF6EBAEC10F09B51E96E050E9C2586
:103E1000EA6EB40EEF6EBAEC10F09B51E96E050E2F
:103E20009C25EA6E6F0EEF6EBAEC10F09B51E96EB6
:103E3000050E9C25EA6E0DC0EFFFBAEC10F099510B
:103E40009B5D0E6E9A519C590F6E0FAE02D0020E02
:103E50000F260FBE06D0E10E0E5C010E0F58D8B033
:103E60002D981200972B04EE00F09751E9266F0E63
:103E7000EF6204D0A6AB02D0A69B396A1200A6B2AC
:103E8000FED717C0A9FF18C0AAFFA69EA69CA680B1
:103E9000A8501200166E14C017F015C018F0EFDF0E
:103EA00016181CE0A6B2FED716C0A8FF14C0A9FFC2
:103EB00015C0AAFFA69EA69CA684F29E550EA76ECC
:103EC000AA0EA76EA682F28EA69414C017F015C093
:103ED00018F0D5DF161802E0D8901200D880120032
:103EE0007FCFF6FF7FCFF7FFF86AA68EA69C08006B
:103EF000F5501200F00ED36EC00E9B6E100E386F90
:103F0000020E396F3A6B110EC26EC16ABE0EC06EE0
:103F1000C00E806E200E926E816AF30E936E616AFF
:103F2000826AFC0E946E200EAC6E900EAB6E100E7C
:103F3000B86E3B0EAF6E0A6A0B6A2B0EC26EC2B22F
:103F4000FED7030EC4140B6EC3CF0AF0220E0A5C18
:103F5000010E0B580BE2899E640E146ECDEC12F02C
:103F6000898E640E146ECDEC12F0E5D70FEE37F0AB
:103F7000ED6AEA50FDE1E950FBE1EF6AF26AF16AAD
:103F8000F06A9D6AA06A9F6AA26AD59ED66A340EBC
:103F9000CD6E9E909D90BA6A300EB16EA68EA69C94
:103FA000F66AF76AF86A0EEE00F0400E0E6E09002F
:103FB000F552F5CFEEFF0E2EFAD70E6A12800EEEF6
:103FC00000F00E50E926EFCF0FF00DDA106E0F5013
:103FD000106212900E2A070E0E64F1D712B01CD098
:103FE0000E6A080E0E600BD00E50FDD90F6E0EEE4D
:103FF00000F00E50E9260FC0EFFF0E2AF2D7BDD910
:104000000BE2899E960E146ECDEC12F0898E960E00
:10401000146ECDEC12F0F3D70D019283130EC26E25
:104020000F01C2B2FDD7030EC4140D6EC3CF0CF046
:10403000010E0C5C030E0D5802E3D8801200D890DC
:104040001200C80E146ECDEC12F007EE00F00A6AF2
:104050000B6A0AC017F00BC018F011DFEE6E0A2AC7
:10406000000E0B22980E0A5C010E0B58F2E30AC7F1
:1040700060F00BC761F00CC762F0602B000E61238B
:10408000622360C00AF707010B6B61C00BF70C6B72
:1040900062C00CF70D6B0A0E0E6E0F6A0EC014F0A4
:1040A0000FC015F000016051F5DE0E2A000E0F2240
:1040B0000EC014F00FC015F06151ECDE0E2A000E98
:1040C0000F220EC014F00FC015F06251E3DE3F0E58
:1040D000070104150101616F05C760F1130EC26E7F
:1040E0000001C2B2FDD7030EC414136EC3CF12F089
:1040F000829782958293200E125C010E135802E281
:10410000828317D0220E125C010E135807E3800E33
:10411000125C010E135802E282850BD0820E125CF3
:10412000010E135806E3800E125C020E1358D8A03D
:10413000828782B504D082B702D082A38283120024
:1041400027EE12F0156A020E156027D0010E146ECC
:1041500002EE1CF01550E926EF6A02EE08F0E9269F
:10416000EF6ADFAC07D002EE08F01550E9261450D4
:10417000EF1209D0DCAE06D002EE1CF01550E92695
:104180001450EF12DD50D8901436080ED926000EC8
:10419000DA221466E6D7152AD6D7200E926E030EC1
:1041A000936EC00E946E156A02EE08F01550E92663
:1041B000EFAE9290EFBE928002EE08F0E926EFAAF1
:1041C0009292EFBA928202EE08F0E926EFA692945C
:1041D000EFB6928402EE08F0E926EFA29296EFB2D3
:1041E000928602EE08F0E926EFA49394EFB493844C
:1041F00002EE08F0E926EFA09396EFB0938602EE68
:1042000008F0E926EFAC9490EFBC948002EE08F041
:10421000E926EFA89492EFB89482010E156E02EE93
:1042200008F0E926EFAE9398EFBE938802EE08F00F
:10423000E926EFAA939AEFBA938A02EE08F0E926EC
:10424000EFA6939CEFB6938C02EE08F0E926EFA25E
:10425000939EEFB2938E02EE08F0E926EFAC9494B1
:10426000EFBC948402EE08F0E926EFA89496EFB82C
:10427000948602EE08F0E926EFA49498EFB49488AF
:1042800002EE08F0E926EFA0949AEFB0948A1200AB
:1042900027EE11F0136A0201020E13603ED0010EE8
:1042A000156E146ADFCF16F0020ED926000EDA2240
:1042B000DFCF17F01738070B176E16BC04D0040AAF
:1042C00002E015501412D8901536060ED926000EAD
:1042D000DA221566E7D7070109A11CD0900E132436
:1042E000E96E080EEA6AEA22EFCF12F002EE10F051
:1042F0001350E92614501214EF6E02EE08F013501A
:10430000E926EF1C126E02EE18F01350E926145045
:104310001214EF6E132A0201BFD708491069120068
:10432000956B126A100E12600CD0080E1202F35038
:10433000100FD96E070EDA6ADA22DF509527122A9B
:10434000F1D7040E01016003F350000195273F0EE1
:10435000951795C006F712007F6A000195517F609E
:104360000BD0A192B368B26AB180A1A2FED7B1907E
:10437000A5B902D07F2AF2D71200020E136EA68EC4
:10438000A69CA684A68EF66AF76AF86AA688550ED9
:10439000A76EAA0EA76EA682A6980A000EEE00F0DF
:1043A000400E146EEECFF5FF0F00142EFBD7550E06
:1043B000A76EAA0EA76EA682A694F66A0EEE00F06D
:1043C0001580400E146E0900F550EE1802E01590AD
:1043D00002D0142EF8D715A002D0D8801200132EC8
:1043E000D0D7D8901200136EFA0FF66E430EF76A0C
:1043F000F722F86A0800F550120000EF02F000EF13
:0244000008F0C2
:0200000400F00A
:1000000017571600270F00E0009F000000000000B7
:100010000020430000000000012043000000000019
:100020000220430000000000032043000000000005
:1000300004204300000000000520430000000000F1
:1000400006204300000000000720430000000000DD
:1000500008204300000000000920430000000000C9
:100060000A204300000000000B20430000000000B5
:100070000C204300000000000D20430000000000A1
:100080000E204300000000000F204300000000008D
:100090000000000000000000000000000000000060
:1000A0000000000000000000000000000000000050
:1000B0000000000000000000000000000000000040
:1000C0000000000000000000000000000000000030
:1000D0000000000000000000000000000000000020
:1000E0000000000000000000000000000000000010
:1000F0000000000000000000000000000000000000
:1001000000000000000000000000000000000000EF
:1001100000000000000000000000000000000000DF
:1001200000000000000000000000000000000000CF
:1001300000000000000000000000000000000000BF
:1001400000000000000000000000000000000000AF
:10015000000000000000000000000000000000009F
:10016000000000000000000000000000000000008F
:10017000000000000000000000000000000000007F
:10018000000000000000000000000000000000006F
:08019000000000000000000067
:020000040000FA
:0400000000EF02F01B
:020000040020DA
:080000001600000000030017C8
:020000040030CA
:0E000000FF280008FF8181FF0FC00FE00F40B6
:00000001FF
